:03000000021BBF21
:0C1BBF0078FFE4F6D8FD7581DD020036E9
:0100190022C4
:0618B6008B318A328933F8
:1018BC007577027F48121A2D121C0BEF20E0F9AB42
:1018CC0031AA32A933120548787FE6FE08E6FDED11
:0118DC00FF0C
:0118DD0022E8
:100F7A0043525354005341564500434647002D3EC1
:100F8A0053320052415445434C5220554E49544223
:100F9A004C4E4B545249475452455653545254534B
:100FAA00544F505A45524F44464C54534156455259
:100FBA00535420535720202E3173202E3273202E63
:100FCA00357320317320203273202035732020316D
:100FDA0030732033307320316D2020326D2020355C
:100FEA006D202031306D2033306D20316820200093
:100FFA0000000100020005000A001400320064012A
:10100A002C025804B00BB8177046508CA046656580
:10101A0074596172644D6574724F6666204F6E2012
:10102A00204E6F2020596573204F66662054696DE3
:10103A0065416C7420547269674F66662054696D05
:10104A0065416C74204F66662054726967507772E6
:05105A00205265632037
:10192C0025E024F9F582E4340FF583220533E53301
:10193C00C394022208F608F608F62275F004A424D3
:05194C0023F9741022D4
:10145100789F76AB0876CD08760008760AE408F620
:1014610008760108F608766408764012194008F6F5
:1014710078ADF608760A08F608763C08F608761480
:1014810008F608760F1219407BFF7A0F797A121845
:09149100007F05121762021860C9
:1018DE00757B1D757CC012156978A0E664CD700409
:1018EE0018E664AB600312145178B9E6FFF4600396
:0718FE00EF700478B97601D8
:0119050022BF
:0D1B8700C2AF7DC07C1DE4FF121AD1D2AFA9
:011B9400222E
:10156900753EFF857B3F857C40754100754200755E
:10157900439FE4FFAB3EAA3FA9408F8275830012C7
:10158900051BAB41AA42A9438F8275830012055AF4
:101599000FBF1CE078B8E6FFF46003EF700478B879
:0215A9007601C9
:0115AB00221D
:101860007D01E4FF1219D57BFF7A0F797F121800F2
:10187000121B87C2AF7F9F7B1C7DC07C1D121ADBB1
:0D188000D2AF7F02121762E4FDFF0219D5FE
:10097A00E4F5317BFF7A0F79841218007F0512178C
:10098A0062A297829650FAA2969217A2979218E5B7
:10099A003175F004A4248DF9740F35F0FA7BFF1237
:1009AA0018007F05121762853132E4F5337BFF7A2E
:1009BA000F7988121800E531B4090050779009CEF2
:1009CA00F82828730209E9020A3E020A0A020A12F0
:1009DA00020A16020A1E020A26020A2E020A367F94
:1009EA0001EF12192C78A1E6FC08E6FD7401936D5B
:1009FA007003E4936C70028F330FBF0FE4020AC1D5
:100A0A0078A3E6F533020AE778A4800278ACE6F523
:100A1A0033020B0178ABE6F533020B2878B5E6F51D
:100A2A0033020B4578B6E6F533020B6278B7E6F582
:100A3A0033020B7FE53165326003020999A2173050
:100A4A009601B35013A296921730960C0531E531F0
:100A5A00C3940C4003E4F531A218309701B350D483
:100A6A00A29792183097CDE531B40C0050C6900A7F
:100A7A007FF8282873020AA3020ACF020AD5020ABB
:100A8A00F3020B07020B1A020B33020B50020B6D17
:100A9A00020B93020B99020B9F0533E533C3940FA4
:100AAA004003753301E53312192CE493FF74019363
:100ABA0078A1CFF608EFF6E53375F004A424BDF962
:100ACA00740F020B8812135B020A3E0533E533C327
:100ADA0094034003E4F53378A3A633E53375F004B1
:100AEA00A42417F97410020B881219384003E4F58C
:100AFA003378A4A633E533121947020B8812193842
:100B0A004003E4F53378ACA633E533121947806E17
:100B1A001219384003E4F53378ABA633E53375F0A0
:100B2A0004A4242BF9741080550533E533C39404C7
:100B3A004003E4F53378B5A633E53375F004A4240D
:100B4A0033F9741080380533E533C394034003E462
:100B5A00F53378B6A633E53375F004A42443F97463
:100B6A0010801B0533E533C394044003E4F533785E
:100B7A00B7A633E53375F004A4244FF9741035F0A1
:100B8A00FA7BFF121800020A3E121451020A3E12A0
:0B0B9A001860020A3E43A208020A3E57
:0A1BD7004552415300444F4E4500B3
:101B470078A1E6F55508E6F55622E56CAE6B780602
:011B5700226B
:10112500C215C21678B9E6C43354E0FEE4F5728EF2
:1011350071F570F56F7B40FAF9F8AF72AD70AC6F71
:101145001206078E698F6AE4F532F533C3E53395E8
:101155006AE5329569501CE53164816016AF33AE9E
:1011650032121832121ABD8F310533E53370DD05A1
:101175003280D9E531B48108E53315337002153273
:10118500E533656A7004E5326569700CD215121B8A
:10119500A3E4F56BF56C800785326B85336CE4F55C
:0911A5006DF56E755480121B47B4
:0111AE00221E
:10183200C3EF956AEE95695024EF7806C333CE3331
:10184200CED8F9FD757702EE787FF6CFEDCFEF08AF
:0D185200F67F50121A7B121C0BEF20E0F9FC
:01185F002266
:031A4800CDEFCD12
:101A4B00757702EE787FF6ED08F67F50121A7B124F
:061A5B001C0BEF20E0F976
:011A61002262
:101ABD007577017F50121A2D121C0BEF20E0F9786B
:031ACD007FE6FFB2
:011AD00022F3
:101AA800121A48E4FFFE0FBF00010EBE0FF8BFA0D8
:041AB800F5121ABD4C
:011ABC002207
:06179800CBEFCBCAEECA44
:10179E00301503301627757703EA787FF6EB08F6D7
:1017AE0008EDF67F50121A7B121C0BEF20E0F9E4C5
:0D17BE00FFFE0FBF00010EBE0FF8BFA0F52B
:0117CB0022FB
:1015EF00753400753500753654E4F533121B51C34D
:1015FF0033CE33CED8F97C002533FFEC3EFEAB342F
:10160F00AA35A93685338275830012051BFD121783
:10161F00980533E533C3940640D2756D00756E0699
:01162F002298
:1011AF008E318F32121B51C333CE33CED8F9256E09
:1011BF00FFE56D3EFEEEC0E0EFC0E0E531FDD0E0B3
:1011CF00FFD0E0FE121798056EE56E7002056D12E6
:1011DF001B51C333CE33CED8F9256EFFE56D3EFEDE
:1011EF00AD32121798056EE56E7002056D0558E564
:1011FF005870020557C3E56E9440E56D9400401793
:10120F00E4F56DF56E056CE56C7002056B956AE59E
:08121F006B95694002D2152213
:10135B00E4F56DF56E7BFF7A1B79D7121800D21668
:10136B00E4F53EF53FC3E53F956AE53E95695021AF
:10137B00E53FAE3E7806C333CE33CED8F9F56E8E4D
:10138B006D7D81FF121798053FE53F70D8053E80B4
:10139B00D4C2167BFF7A1B79DC121800E4F56BF5CF
:0713AB006CF56DF56EC21533
:0113B2002218
:10130200E4F53EF53FF540F541C3E541956AE54018
:1013120095695044E53F6481603EAF41AE4012188A
:1013220032121ABD8F3FE53F64807022AF3E053E08
:10133200FCFDFEFBFAF9120D517F2C120016AE4095
:10134200AF41E4FCFDFBFAF9120D51121BF4054109
:08135200E54170B5054080B1D2
:01135A002270
:02149A008F3E83
:10149C00E4F53FF540F541F542C3E542956AE54177
:1014AC0095695030E5406481602AAF42AE41121814
:1014BC0032121ABD8F40E540B4800FE53F653E7097
:1014CC0007AF42AE41021832053F0542E54270C9F2
:0414DC00054180C581
:0114E00022E9
:10163000121B4778ACE6F559E4F557F5581215EF4B
:10164000856B73856C747F0112129E30021A78AF1D
:10165000E6FE08E6FFE4FCFD7B64FAF9F812057C7F
:101660008F668E658D648C63300505C205121A92F3
:011670002257
:10172800856B31856C32E56E456D60080532E532B2
:101738007002053185736B85746C1215EF85316BFA
:1017480085326CC3E532956AE53195694007E4F561
:0A1758006BF56CD2157F0202129EA1
:101AD100740478FF769612FF0322740078FF7696DD
:041AE10012FF0322CB
:0300330002105F59
:0D105F00C0E0C0F0C083C082C0D075D008D2
:10106C00E5D954F8FF12072010990810991010A810
:10107C001810C32010AA2810C33010C53810CB404C
:10108C0010C34810E4501101580000110F857ADA92
:10109C00C2DDC2DC7578007579008070800EE57752
:1010AC00700280560579E579700205781200268F5A
:1010BC00DAC2DDC2DC80558016D2DDC2DC804DC2C6
:1010CC00DDC2DCE5777004C2DA8041D2DA803DC241
:1010DC00DDD2DC7575048034AFDA121BCB0579E5F3
:1010EC007970020578C2DDC2DCE5777004C2DA8063
:1010FC001BD2DA8017AFDA121BCBC2DDD2DC7575CE
:0E110C00028009757504C2DDC2DCD2DAC2DBD6
:0B111A00D0D0D082D083D0F0D0E032E3
:10188D0043910C43920CE4F5DBEF25E0F5DB3017CB
:10189D000343DB0175DD2575DC2575D84453F8FE52
:0918AD0053F7FEE4F575D2E822C0
:101A7B00E57530E002FF22E4F576757503EF25E09E
:071A8B00F57AD2DD7F022293
:101A2D00E57530E002FF22E4F5761577757505EF63
:0B1A3D0025E04401F57AD2DD7F022293
:061C0B0020DBFDAF752295
:0D0026001577AF760576747F2FF8E6FF2280
:0C1BCB00747F2576F8EFF605761577227A
:0E1B9500E4F5847585FFF592F5A475A5FF2291
:071BFD00EE3395E0FDFC2230
:10195100C212C214C211D2A2C2A0C2A1E4FDFF12DE
:1019610019D5E4FD7F011219D57F0812129E7F045B
:0319710002129EC1
:1019D500EF146011047016BD0104C2A78002D2A7DE
:0E19E500A2A7921322BD0103C2A622D2A622FF
:10129E00EF14B40800505C9012B375F003A4C5832C
:1012AE0025F0C583730212CB0212D10212D802129C
:1012BE00E40212E60212E40212F00212F8D21275E1
:1012CE00190122C212A21392A722D214751A057DF9
:1012DE00017F010219D58005C211C28722C211D227
:1012EE008722D211D28775180122C2A47F0112174C
:0412FE0062D2A422F2
:1016B000301212D5190F30A707C2A775191E800561
:1016C000D2A7751946E51AD39400400CD51A09C261
:1016D00014E4FD7F011219D5301111D5180E308791
:0D16E00006C28775180522D28775181E22D4
:10199500C374039FFE1392A0EEA2E192A1AF80CF84
:0F19A5005480CFED547FCF4FCF8F80C2A2D2A2FC
:0119B4002210
:061800008B408A41894281
:10180600E4FCCFECCF7D201219950CBC04F4E4FC6B
:10181600AB40AA41A9428C8275830012051BFD606C
:0B1826000ACFECCF1219950CBC04E5B2
:011831002294
:041227008F828E83A1
:10122B00121BFDE47B0F7A27F9F8C31206A75003B4
:10123B0090270FAF82AE83121BFD7B197AFC79FFCF
:10124B0078FFD31206A7400390FC19E4F531741B09
:10125B002531F8E4F60531E531B405F2AE83AF8202
:10126B00121BFD7B007A00791B120D51E51E701AC3
:10127B00753103741A2531F8E6FF741B2531F8C656
:10128B00EFC6D531EE751B2080E27B007A00791B0F
:03129B0002180036
:1019F30046554C4C0050524F47005A4C4F47004DF0
:0D1A03004F440076322E380054726967009F
:101B2100E6FE08E6FFE4FCFD2278D61206E278CE56
:031B31000206FBAE
:030013000219745B
:10197400C0E0C0D075D010200E0CAF8DEFAD8BF54C
:101984005EEDF55FD20E758D00758B00D0D0D0E082
:011994003220
:021762008F3FB7
:10176400E4F540F541C3E541953FE540940050233D
:10177400900000AF82AE83E4FCFD7B207A4EF9F842
:10178400D31206A74003A380EA0541E54170D605BC
:031794004080D2C0
:01179700222F
:0E1BA3007BFF7A1979F31218007F0A0217628D
:0F1B6900D20B301506121BA3C20B22121630220C
:05000E00C20B021728DF
:101A920078DA12070700000000121B2A78D6120714
:061AA20007000000002215
:10003600121B95121BE11219517F041217622097A9
:10004600127BFF7A1979F81218007F011214E1D297
:10005600AF80FE209612D2AF1218DEC2177F701242
:10006600188D12112512097A7A1979FD1204F7E40E
:10007600FF1214E1D2AF1218DE7BFF7A1A79021250
:10008600180078B8E62430FD7F031219957F041214
:1000960017627A1A79061204F7C2177F7012188D42
:1000A6007F01121762121125120019C21A1216EDDB
:1000B6007F01121762E4F560F56112001AA29692AA
:1000C60008A2979209E4F52478D2120707000000E7
:1000D60000E4F52578DA120707FFFFD8F178CE128B
:1000E600070700000000E4F55378D6120707000062
:1000F6000000C20DC20BC20CE4F567F568F526F5E3
:1001060027F55EF55FC20EF562C20FF55DF55CF58B
:100116005BF55AF566F565F564F563F52078B5E6A1
:1001260024FE600B14600C2402700AD2018006D2F1
:10013600068002D20078B6E624FE6007047006D276
:10014600028002D20778B7E624FE600B14600C2406
:1001560002700AD2038006D2048002D2053001174B
:10016600C20178AD121B217B64FAF9F812057C8F67
:100176005D8E5C8D5B8C5A301AFDC21A300C33A230
:1001860008309601B3400BA209309701B340030231
:10019600026430961230970FC20CE4F567F5687F5B
:1001A6000412129EE4F553A2969208A297920902AF
:1001B6000264209605209702D21030965630975347
:1001C600301031C21078CE1206E2EC4D4E4F78DA7E
:1001D600700C12070700000000121B2A801012077D
:1001E600070000000078CE12070700000000D209C1
:1001F600D208802478A4E6601F0568E568700205C9
:1002060067D394B8E567940B400ED20C7F051212A3
:100216009E8005E4F567F568A208309601B3501F85
:10022600A2969208309618201015C201E553600771
:10023600E4F5537F0680057553017F0712129EA2CF
:1002460009309701B35017A29792093097102010E2
:100256000DB20B300B05121B69800312000E12073C
:1002660046AF5DAE5CAD5BAC5AEC4D4E4F6026744E
:10027600FF2FF55DEE34FFF55CED34FFF55BEC34F6
:10028600FFF55AAF5DAE5CAD5BFC4D4E4F70062080
:100296000B03121B69AF66AE65AD64AC63EC4D4EE5
:1002A6004F602374FF2FF566EE34FFF565ED34FFDE
:1002B600F564EC34FFF563AF66AE65AD64FC4D4E98
:1002C6004F700312000E200E03020374C2AFC20E5B
:1002D600D2AFE4855F30855E2FF52EF52DAF30AEBB
:1002E6002FAD2EAC2D7B107A27F9F812057C8F30B6
:1002F6008E2F8D2E8C2DE4FB7A90F9F81215258F12
:10030600308E2F8D2E8C2D78ABE66009C374B89F86
:10031600FF740B9EFEE56214601624FE6020240323
:100326007049C3EF94B0EE9404500E7562018009D3
:10033600D3EF9414EE940540357562038030C3EF15
:1003460094B0EE94045027756201300006200B032A
:10035600121B69300305C203121A92300B02D20F28
:100366007BFF7A1A790B1218008003E4F5620525E3
:10037600E525C3940250030204F1E4F525FB7A0057
:1003860079281218B68E298F2AE52864026003029E
:1003960004F178D21206EEE8C0E0E9C0E0EAC0E077
:1003A600EBC0E078A3E6FDAF2AAE29121405D0E033
:1003B600FBD0E0FAD0E0F9D0E0F8EB2FFFEA3EFE02
:1003C600E93DFDE83CFC78D21206FB0524E524C392
:1003D600940550030204F178D21206E2E47B05FA92
:1003E600F9F812152578D21206FB78D21206E278B1
:1003F600CE1206EEC3EF9BFFEE9AFEED99FDEC984A
:10040600FC78D21206FB78DA1206E278D21206EEF1
:10041600D31206A7400A78D21206E278DA1206FB51
:10042600E553600A78DCE6FE08E68E2BF52C78D4D8
:10043600E6FE08E68E29F52AE5536006AF2CAE2BBC
:100446008004AF2AAE291212270527E52770020578
:1004560026C378A296E52618964040E4F526F527A9
:10046600300D0DE529FF120016AF2AE52A120016F7
:10047600300B287F0312129E20151A78ACE6600C0A
:10048600300F097F007E821211AFC20FAF2AAE294C
:100496001211AF8006121BA312000E78D21206E2CA
:1004A60078D61206FB78D212070700000000E4F5A2
:1004B60024300405C204121A9230061678B1121BB3
:1004C6002178D61206EED31206A74006200B031299
:1004D6001B6930071678B3121B2178D61206EEC3B5
:1004E6001206A75006300B0312000E1216B00201B8
:0104F6007D88
:0B04F7007BFF1218007F041217622226
:10190600444C0021536967005A4C4F47004D4F44E1
:1019160000322E38004665622031352032303035AF
:061926000050524F470083
:1015AC00AF39AE38AD37AC36EC4D4E4F22EF24FF91
:1015BC00F539EE34FFF538ED34FFF537EC34FFF543
:1015CC003622E475392075384EF537F53622E47538
:1015DC003901F538F537F536227533007534007559
:0315EC00359F2206
:0F1B78007F0412129EE4F553C20CF567F5682244
:10074600121BB1EF700302095A121A10EF1207209A
:1007560009352409412A094750088D52077E610848
:100766000F6308626C08687208657308917409055E
:100776007608FF780000095A121B787BFF7A1979F0
:10078600061218001215CE121BB1EF700A1215AC24
:1007960060051215B980F01215AC700302095A12E1
:1007A6001A108F3212149AE4F5391215DEE47F0618
:1007B600FEFDFCAB39AA38A937A836C31206BD50D0
:1007C6001F121ABD8F32120016E5392401F539E4DD
:1007D6003538F538E43537F537E43536F53680CD36
:1007E600121ABD8F32E53264806016E5326481608C
:1007F60010120016121ABD8F3212001675310180C2
:1008060003E4F531E53170D8221215E51215DAF553
:10081600321215AC60241215CE121BB1EF700A12FB
:1008260015AC60051215B980F01215AC60031209FB
:100836005B0532E532C3941C40D71215AC601A78BA
:100846009FB6AB0708B6CD0302093E7BFF7A19793E
:10085600091218007F0A0217620208FCB20D220272
:1008660013021215E5E4F532AB330535E535AA3446
:100876007002053414F9120502FF1200160532E55E
:1008860032C3941C40E22243A20822121B7875331D
:100896000075340075357D1215DAF5321215AC6027
:1008A600241215CE121BB1EF700A1215AC60051298
:1008B60015B980F01215AC600312095B0532E532FA
:1008C600C3940240D71215AC602CAE7DAF7EEE33DA
:1008D60095E0FDFC78D61206EEC3EF9BF53DEE9A49
:1008E600F53CED99F53BEC98F53AAF3D78A9E53C3A
:1008F600F608EFF68042021569121B7802135B7A3E
:1009060019790E12096F7A197913121B3478B8E621
:100916002430FF120016121BF47F761200167A1985
:10092600791712096F7A19791B121B34021BF412FC
:100936001B78E478A9F608F6021860121B780214F0
:1009460051121B787BFF7A1979271218007F011242
:0409560014E180FE2A
:10095A0022121A10AB33AA34A93585328275830064
:10096A00EF12055A227BFF121B34121BF47BFF2263
:0A1BE100E4F5955396BF53A27F224E
:1016ED005389F0438901538FFE758C70E4F58A534D
:1016FD00B8FD53B7FDD2A9D28C53890F43899053AE
:10170D008FEFF58DF58B4391105392EF53B8F7533F
:0B171D00B7F7D2ABD28ED28AD2AA223C
:03000B00021BEBEA
:091BEB00D21A758C70758A003263
:03001B00021C04C0
:071C0400758D00758B0032A5
:101AE5000D0A003031323334353637383941424307
:041AF500444546001E
:101AF900AF52AB46AA47A948055222AF45AE44ADFD
:041B090043AC422285
:1014E1005387BF75985053877FE4F5BABF01054311
:1014F100A240800353A2BFE4F5BD75BE30F5BF75B0
:10150100BD035391FE4392014391025392FDC21BCD
:1015110053B8EF53B7EF43B81078CCF618F678CD3F
:04152100F6D2AC2230
:030023000217CCF5
:1017CC00C0E0C0D075D01030981E78CCE6C3940F12
:1017DC00501418E60624BBF8A69978CC0618E6C374
:1017EC00941040027600C298309904C299C21BD062
:0417FC00D0D0E03237
:08000300201BFDD21B8F992286
:1019B50078CCE6D39400401508E60624BBF8E6FF8C
:0F19C50078CC1608E6C394104005E4F6227F00A4
:0119D40022F0
:03001600020003E2
:101A10007F207E4E78CCE67010D3EF9400EE9400D9
:0C1A20004007EF1F70EE1E80EB1219B59E
:011A2C002297
:101B3400120502FF600C120016740129F9E43AFA46
:031B440080EE220E
:0E1BB10078CCE6D3940040037F01227F00220F
:101A6200CEEFCEEE54F0C4540F901AE893FF12005A
:091A720016EE540F93FF0200165A
:101B5800CDEFCDCCEECCEEFF121A62CFEDCF021A4C
:011B6800621A
:091BF4007BFF7A1A79E5021B342B
:0E0D51008F458E448D438C428B468A478948DD
:100D5F00E4F552EC4D4E4F7017E94A4B70057F305A
:100D6F00020016121AF98F827583007430020E7406
:100D7F00121B06EC33502AE5484547454670077F5E
:100D8F002D120016800D121AF98F82758300742DA3
:100D9F0012055A121B041206998F458E448D438CEF
:100DAF0042755101754C00754BCA754A9A75493B8E
:100DBF00E4FFFEFDFCAB4CAA4BA94AA849D312068F
:100DCF00BD5003020E5F121B04A8491206078F5075
:100DDF008E4F8D4E8C4DEC4D4E4F7004E551702360
:100DEF00E5502430FFE5484547454670051200168B
:100DFF00800EAE52121AFB8E82758300EF12055AC7
:100E0F00E4F551AF4CAE4BAD4AAC49AB50AA4FA92C
:100E1F004EA84D12057CC8ECC8C9EDC9CAEECAC3AD
:100E2F00E5459FF545E5449AF544E54399F543E5D6
:100E3F004298F542AF4CAE4BAD4AAC49E47B0AFA4F
:100E4F00F9F81206078F4C8E4B8D4A8C49020DBF55
:100E5F00E547454845466010AB46AA47A948855225
:080E6F0082758300E412055AAC
:010E77002258
:100BA5000134C35001DBBF68028BBB800344B79897
:100BB5000407B3B004D5AFC805A9ABE00689A7F80B
:100BC5000775A410086DA02809719C400A819858E2
:100BD5000B9F94700CCA90880DE98CF90E048CA0BB
:100BE5000EA88AAC0F4D88B80FF786C410A184D023
:100BF500115182DC120580E812BB7EF413747D006E
:100C050014307B0C14F2791815B8772416807530DA
:100C1500174B733C1819714818ED6F5419C46D6062
:100C25001AA16B6C1B7E69781C6167841D4A6590EF
:100C35001E37639C1F2561A8201A5FB421125DC071
:100C4500220D5BCC230E59D8241557E4251F55F0EA
:100C5500262F53FC27425208285B501429764E2034
:100C65002A9B4C2C2BC04A382CEE48442E1E46504D
:100C75002F55445C308F426831D1407433173E8024
:100C850034633C8C35B13A98370938A4386636B0A8
:100C950039C734BC3B2D32C83C9D30D43E0F2EE0C5
:100CA5003F882CEC41062AF8428D29044418271068
:100CB50045AB251C4741232848E121344A861F407E
:100CC5004C311D4C4DE21B584F9C1964515D1770FA
:100CD5005323157C54EF138856C4119458A20FA0C2
:100CE5005A830DAC5C6D0BB85E6009C4605807D0C3
:100CF500625A05DC646203E8667301F4688A0000E1
:100D05006AA1FE0C6CB8FC186ECFFA2470E6F830B8
:100D150000000000000000000000000000000000CE
:100D250000000000000000000000000000000000BE
:100D350000000000000000000000000000000000AE
:0C0D4500000000000000000000000000A2
:1016710075F004E538A424A5F582E5F0340BF58373
:10168100E49322FE740193FF75F004E538A422F57A
:1016910083C37401939FFFE4939EFEE4228F398EEE
:0F16A100388D378C36228F358E348D338C322234
:101B0D00C3EF9DEE9C400AD3EF9BEE9A50037F01ED
:041B1D00227F002201
:040E78008E368F37EC
:100E7C00E4F538121671FC740193FD12168924A93D
:100E8C00F582E5F0340BF583E493FA740193FBAF30
:100E9C0037AE36121B0DEF7003020F68121671126B
:100EAC00168424A9F582E5F0340B1216908F3C8E33
:100EBC003BF53AF53912168924ABF582E5F0340B83
:100ECC00F583E49312168424A7F582E5F0340B1213
:100EDC0016908F408E3FF53EF53DAD3EAC3D120673
:100EEC00998F408E3F8D3E8C3DAE36AF37E4FCFD86
:100EFC00EEC0E0EFC0E0121671FE740193FBCAEE77
:100F0C00CAD0E0FFD0E0FEC3EF9BFFEE9AFEED945B
:100F1C0000FDEC9400FCAB40AA3FA93EA83D120595
:100F2C007CAB3CAA3BA93AA839121525C8ECC8C918
:100F3C00EDC9CAEECACBEFCB12168924A7F582E510
:100F4C00F0340BF583E493FE740193FFE4FCFDEBAA
:100F5C002FFFEA3EFEED39FDEC38FC220538E53872
:0D0F6C00C3946A5003020E7FE4FFFEFDFCFB
:010F79002255
:01001A0022C3
:1013B30012169EAB39AA38A937A836E8C0E078A739
:1013C300E6FE08E6FFE4FCFDD0E0F812057C121609
:1013D3009E780E1206CE12169E78A9E6FE08E6FF48
:1013E300EE3395E0FDFCE5392FF539E5383EF53868
:1013F300E5373DF537E5363CF536AF39AE38AD3731
:02140300FC22C9
:021405008D3127
:10140700120E781216A71213B31216A7E53114603D
:101417001C14702DE47FE87E03FDFCAB35AA34A9CC
:1014270033A83212057CE47BE87A0B800CAF35AE2B
:1014370034AD33AC32E47B03FAF9F81215251216F2
:09144700A7AF35AE34AD33AC3271
:011450002279
:10050200BB010689828A83E0225002E722BBFE02F7
:09051200E32289828A83E493222A
:10051B00BB010CE58229F582E5833AF583E0225095
:10052B0006E92582F8E622BBFE06E92582F8E222DF
:0D053B00E58229F582E5833AF583E49322F9
:10054800BB010689828A83F0225002F722BBFE0192
:02055800F3228C
:10055A00F8BB010DE58229F582E5833AF583E8F0D7
:10056A00225006E92582C8F622BBFE05E92582C883
:02057A00F2226B
:10057C00E88FF0A4CC8BF0A42CFCE98EF0A42CFC1E
:10058C008AF0EDA42CFCEA8EF0A4CDA8F08BF0A49C
:10059C002DCC3825F0FDE98FF0A42CCD35F0FCEBFB
:1005AC008EF0A4FEA9F0EB8FF0A4CFC5F02ECD39C0
:0F05BC00FEE43CFCEAA42DCE35F0FDE43CFC222D
:1005CB0075F008758200EF2FFFEE33FECD33CDCCE7
:1005DB0033CCC58233C5829BED9AEC99E58298406A
:1005EB000CF582EE9BFEED9AFDEC99FC0FD5F0D647
:1005FB00E4CEFBE4CDFAE4CCF9A88222B800C1B971
:10060B000059BA002DEC8BF084CFCECDFCE5F0CBAE
:10061B00F97818EF2FFFEE33FEED33FDEC33FCEBE7
:10062B0033FB10D703994004EB99FB0FD8E5E4F9A2
:10063B00FA227818EF2FFFEE33FEED33FDEC33FC8F
:10064B00C933C910D7059BE99A4007EC9BFCE99A83
:10065B00F90FD8E0E4C9FAE4CCFB2275F010EF2FC8
:10066B00FFEE33FEED33FDCC33CCC833C810D707C8
:10067B009BEC9AE899400AED9BFDEC9AFCE899F803
:0E068B000FD5F0DAE4CDFBE4CCFAE4C8F92296
:10152500C2D5E830E70FB2D5E4C39BFBE49AFAE4F1
:1015350099F9E498F8EC30E717B2D512155B120665
:1015450007E4C39BFBE49AFAE499F9E498F880036D
:1015550012060730D50DE4C39FFFE49EFEE49DFD12
:04156500E49CFC22E4
:0E069900C3E49FFFE49EFEE49DFDE49CFC2272
:1006A700EB9FF5F0EA9E42F0E99D42F0EC6480C8CA
:0606B70064809845F0226A
:1006BD00EB9FF5F0EA9E42F0E99D42F0E89C45F093
:0106CD00220A
:1006CE00E86010ECA2E713FCED13FDEE13FEEF1342
:0406DE00FFD8F0222F
:0C06E200E6FC08E6FD08E6FE08E6FF2244
:0D06EE00E6FB08E6F908E6FA08E6CBF8227C
:0C06FB00ECF608EDF608EEF608EFF6222B
:10070700D083D082E493F608740193F608740293B9
:09071700F608740393F6740473F0
:10072000D083D082F8E4937012740193700DA3A368
:1007300093F8740193F5828883E47374029368607C
:06074000EFA3A3A380DF7C
:00000001FF
